:020000040000FA
:020000003428A2
:08000800A100030EA2000B1180
:100010009C0A20141C08FF3C031D2F289C01A014DF
:10002000AB0A2B08FB3C031D1728AB012F2802301D
:10003000050685059D0A1D083C3C031D2F289D01D2
:1000400020159E0A1E083C3C031D2F289E01A0156A
:100050009F0A1F08183C031D2F289F012016220EFF
:1000600083002108090034288B0185010A308600AD
:100070008316F8308500F0308600833081008312CB
:100080000000000094011414000000309F000030B4
:100090009E0000309D00A0308B0050284D28342851
:1000A000A0103C21A01C7928A0105421A01C7B2862
:1000B000A0104321A01C7E28A0105421A01C802841
:1000C000A0104821A01C8328A0105421A01C852822
:1000D000A0104F210515A01C8828A0105421A01C99
:1000E0008A28A0105421A01C8D28A010051150288A
:1000F00008009020522890205721562890205A28F6
:10010000902057215E289020622890205721662851
:1001100090206B28902057216F289020572173281A
:1001200011219A1895209A01080005159001910156
:10013000A6012608022111219A18AB281A19A22813
:100140009A019928A60A2608033C031DA928A6019E
:10015000A0282608A02890011008022111219A1831
:10016000C9281A19B5289A01AC282608023C031D93
:10017000C228BB28B328900A1008043C031DBA28E3
:100180009001BA28900A10080A3C031DBA28900171
:10019000BA28A7012708022111219A18DA281A196A
:1001A000D3289A01CA28A70A2708063C031DD92884
:1001B000A701D12891011108022111219A18EB28D9
:1001C0001A19E4289A01DB28910A11080A3C031D38
:1001D000E2289101E22826080319F32810080A3EB4
:1001E0009000A60BEB2810089F0027080319FD2894
:1001F00011080A3E9100A70BF52811089E009D01E9
:10020000051108005F210F3986000800201C06290F
:100210002010A30A2308063C031D0629A301080099
:1002200034289A01061A19291A140621060E9A056D
:100230002D29861A20299A140621060E9A052D29A1
:10024000061B27291A150621060E9A052D29861B3D
:100250002D299A150621060E9A05080034281D0836
:100260005F2192001E085F2191001F089000482125
:100270003A210800860008001F085F219000100E38
:100280000F39860008001F085F210F39860008001B
:100290001E085F219100110E0F39860008001E080C
:1002A0005F210F39860008000A30860008001C080C
:1002B0005F218C008C0E0C080F398600080093011A
:1002C000F63E031C6529930A60290A3E930E9304A7
:1002D0001308080034280D08C6308C000000000008
:0C02E0008C0B6E298D0B6C290800342853
:084000000400010005000500A9
:02400E00F93F78
:00000001FF
